:020000020000FC
:100000004BCDA4C1000000001FC000008DC0000047
:10001000000097C00000000000000000020304067A
:10002000080C10182030406080000406080C1018DE
:100030002030406080A0C0000003070F1F000505AE
:100040000D050305030302004FB662FD0CC05520E9
:1000500041F00994C52DC095089483FDC795C4BD92
:1000600064604FBE1895C0916400089483FDC795E5
:10007000C4BD6B7FC0916400CF3F09F41EC070FF08
:100080001AC082FD05C04FBE9598AC98C0981895CF
:1000900076FD0EC065FD0CC0C091B100C0FD949806
:1000A000C1FDAD98C2FDAB98CAEFC095CA95F1F7F6
:1000B0009598AC98C0984FBE189524BCCC27C064C6
:1000C000C8BF6460F8CFC6CF70FFC4CF65FDC2CF94
:1000D000959AC0CF70FFBECF65FDBCCFAC9ABACFAA
:1000E00070FFB8CF65FDB6CFC09AB4CF949A70FFB9
:1000F000B1CF65FDAFCFC7E0CA95F1F7959AAACF0A
:10010000AD9A70FFA7CF65FDA5CFC7E0CA95F1F7FF
:10011000AC9AA0CFAB9A70FF9DCF65FD9BCFC7E097
:10012000CA95F1F7C09A96CF4FB6C9B7CF7EC9BF6F
:100130006E7FCCB5CE0DDDB5DF1DDBBDCABD4FBEBC
:1001400018953FB68F7EABB7A074A2118061A0E076
:10015000ABBFA9B7AE7FA9BF7894A0916800AA23CE
:1001600041F085FD2AC0A0916800AA95A09368007F
:1001700024C040E050E085FD14C0A0B396FDA095DA
:10018000A2FD4FEFA3E096FDA2E0A5BFAA27A064C1
:10019000AABF8D7FA0B396FDA095A2FD5FEF451786
:1001A00041F7A8E161FDA093680085FD03C0A8E1C7
:1001B000A093680040939600816085FD0EC0A091D9
:1001C0006900AA2331F0A0916900AA95A093690063
:1001D00004C08061AA27A064AABF80FF3DC0A0918F
:1001E00096004A2F61FF8E7F85FD18C0403F08F0C2
:1001F00040EFA42FA295AF704A0F5091B600533034
:1002000069F0A695A69550FD01C0A69552FD03C0C4
:10021000A41B4A2F03C04A0F08F44FEFA0919F0080
:100220004A1708F44A2F40936100A72FA670A1F047
:1002300073FD12C0A0917000AA0FAA0F50919E00EA
:1002400056955695541708F0452F4A0F4093610074
:1002500018F4AFEFA0936100A0916100A093630038
:1002600040916300A0919B004A1708F04A2F542E3A
:10027000A091A000AA2309F422C0542F5A1B10F405
:10028000A42F50E0BA2E8894AA1FAA2EA091A200F3
:10029000A095AA22A50E58F0A091A100A21509F0E0
:1002A000AA95AA0EA093A10048F04A2D08C0A091DB
:1002B000A100BA1608F0A395A093A1004FEF4093B8
:1002C00064007F7B485F08F07064A52DA03408F0BF
:1002D0006860A0916000A395A093600051F0F8942D
:1002E000A9B7A160A9BF84FF02C0A0E4ABBF3FBE15
:1002F0001895A0917400A395A093740041E05091CB
:100300006800552329F085FF03C05A955093680073
:10031000A0919600A13018F0209299000DC0209273
:100320009A002092A300A0919900AF5FA09399003A
:1003300018F0AFEFA0939900F894A9B7A160A9BFF6
:1003400084FF02C0A0E4ABBF3FBE18953FB64CB5DA
:100350005DB58F7EABB7A074A2118061A0E0ABBF8A
:10036000A9B7AE7FA9BF789481FD23C0A2E096FD16
:10037000A3E0A5BF8260A0B396FDA095A2FF05C033
:1003800040936500509366003EC1A3E096FDA2E055
:10039000A5BFAA27A064AABF8D7F85FF01C026C183
:1003A00040E0A0B396FDA095A2FD20C14093960029
:1003B0000FC1A3E096FDA2E0A5BF8D7F61FF71C0D4
:1003C000A2E096FDA3E0A5BFAA27A064AABF826011
:1003D0004093910050939200A0908F004A19B090E2
:1003E00090005B09BB24A22C4C38520518F42092D3
:1003F000950049C0A091D400AA2359F1483C520568
:1004000028F4A0E1BA2EAAE0AA2E23C04836A1E023
:100410005A0728F4A8E0BA2EAFE0AA2E1AC0403D31
:10042000A2E05A0728F4A4E0BA2EAEE1AA2E11C029
:10043000403AA5E05A0728F4A2E0BA2EACE3AA2E6F
:1004400008C04839A8E05A0720F4A1E0BA2EA8E76E
:10045000AA2EC42EA0919300CA1AD52EA091940062
:10046000DA0ADD202AF4AFEFC094D094CA1ADA0A6F
:1004700020929500A8E0A210A0E0CA14DA0618F4B1
:10048000A1E0A09395004093930050939400409175
:1004900091005091920040938F005093900042E061
:1004A00097C0A09165004A1BA09166005A0B94FD6D
:1004B00082C093FD80C092FD7CC086FF03C0D52E14
:1004C000C42E0CC05695479591FD73C0569547951F
:1004D00090FD6FC0D52EC42ED694C79461FD19C06F
:1004E000AC2DAC51AD2DA24008F005C0DD2089F443
:1004F000AC2DA85C70F4A0916700A395AA2311F01D
:10050000A0936700AA3008F471C020929600816021
:100510006DC0A0916700AA2319F0AA95A093670067
:10052000A22C5091BA0097FD06C0A090C80053308D
:1005300011F4A090D000AAEFAA0EA22DA21DCA18F5
:10054000DA0A4FB74170533049F4442321F087FD54
:1005500005C0806803C087FF01C08F77442359F02E
:10056000533031F4AFEFC094D094CA1ADA0A03C002
:1005700040E050E020C0533049F4CC0CDD1CAAE030
:10058000CA1AD20818F4A0E0CA2ED22CAFEFCA16AD
:10059000D20418F04FEF50E00EC0A091AC00CA9EFC
:1005A000412D000C441F50E008F012C04FEF50E006
:1005B0000FC05695479594FF07C0552309F04FEF9C
:1005C000A42FA6954A0F521D4F3F520508F04FEF3A
:1005D00040939600816061FF09C0AFE1A095A92317
:1005E000AB299A2F8F7DBB2009F48062A8E1A093EC
:1005F000680085FF03C0AAE0A093680061FD03C006
:1006000085FD01C08F7E85FD03C0A6E0A093690033
:10061000F894A9B7A160A9BF84FF02C0A0E4ABBF52
:100620003FBE189511E00AC013E008C01AE006C0EA
:100630001EE104C014E602C018EC00C005E1BB27AF
:10064000BA95F1F70A95D9F71A95C1F708952AE3F3
:1006500038E709C020E33CE806C02AE234EB03C0D7
:1006600025E238EC00C012E0BB27AD9ABA95F1F74D
:10067000AC9ABA95F1F7AC98BA95F1F7AD98BA95EE
:10068000F1F7123009F0959A123009F4C09AB0913E
:10069000AD00BA95F1F7123009F09598123009F4CF
:1006A000C098B7E8BA95F1F71A95F1F6022FB22F74
:1006B000BA95F1F70A95D9F73A95A9F6AD9A089542
:1006C000221B39E0001F3A9509F40895221F211BCF
:1006D00018F4210F8894F6CF0894F4CF622C722C72
:1006E000B0E08894B395221F331FE0F73795279524
:1006F0008894912E802E020B130B10F4192D082DC7
:1007000010F4889401C00894661C771CBA9571F7A0
:10071000172D062D0895322D11232AF43A950095B0
:100720001095031B130BF894029F712C002D129F40
:10073000912C802C7894780C172D921C292DB4E0E4
:100740006B2E2695179507956A94D9F7332321F0D8
:1007500000951095031B130B0895089510917B00CD
:10076000169500917A000795B0917E00B01B0B2F73
:10077000B0917F00B10B1B2F28F40038BFEF1B078F
:1007800040F009C00F37120508F405C00FE710E06C
:1007900002C000E81FEF00938300109384000895C7
:1007A00000918300B09180000B0F10918400B091F4
:1007B00081001B1F20E03091840033230AF42A9526
:1007C000B09182002B1F1AF4203F40F00AC02F3056
:1007D00008F407C00FEF1FEF2FE003C000E010E0A8
:1007E00020EF30916300B0919B003B1718F432303A
:1007F00030F009C0B0918400BB235AF004C0B0911E
:100800008400BB2332F40093800010938100209376
:10081000820008952091D70000918300000F10916D
:100820008400111F78DF11232AF40038BFEF1B0763
:1008300040F009C00F37120508F405C00FE710E0BB
:1008400002C000E81FEF002352F0B0916200B01B1D
:100850000B2F18F0013008F00AC001E008C0009525
:100860000F5FB09162000B0F08F001C00FEF009313
:10087000850008952091D800009181001091820098
:100880004ADF11232AF40130BFEF1B0740F009C0F3
:100890000F3F120508F405C00FEF10E002C001E0A1
:1008A0001FEF112352F0B0918500B01B0B2F18F0F1
:1008B000013008F00AC001E008C000950F5FB09158
:1008C00085000B0F08F001C00FEF0093630008953F
:1008D0000FEF677F71FD29C072FD09C06860B0919C
:1008E0007B00BA3020F0B52DB03408F4677FB091AA
:1008F000D300BB23D1F0B0917B00BB23B1F00FEF4D
:1009000010917B00DDDEF894B091730072FDB5E0CC
:100910000B9F112D002D7894112309F00FEFB0914A
:100920009E000B1710F400919E0000939D00089507
:1009300000917A0010917B0000541140B0919D000D
:1009400010F4BA9501C0B39511F0B0939D000895CD
:1009500000C008952091B500B6B1B6FDFBCF04B13B
:1009600015B1B6B1BF77B6B9B091AA00B395B0933F
:10097000AA00B83060F12092AA00B091D200BB2347
:1009800021F1112329F0B091AB00BF3F61F009C004
:10099000B091AB000B1739F020F4BB2321F0BA95CE
:1009A00002C0B395E1F300919B00B093AB00B8385F
:1009B00050F400ECBD3738F400E8B23720F400E41E
:1009C000B73608F400E000939B007F7E0895B09155
:1009D0009B00B39511F0B0939B00B091AA00B73083
:1009E00009F47061089502E3F894B091D9000B9F67
:1009F000012D000C001F7894B0919B000B1710F094
:100A000000919B000093610000936300502E0093BF
:100A1000640000939E00089520927A00B0EFB09396
:100A20007B000895F8940CB51DB52091740078945E
:100A300030917500609076000093750010937600F9
:100A4000031B160971FD03C077FD7DC027C07090A0
:100A50007700209377002709222311F00FEF1FEF73
:100A600080907800909079003093780060927900BF
:100A700000917500109176000819190920917A00EB
:100A800030917B0036952795020F131F10F40FEF5E
:100A90001FEF00937A0010937B0029C020917A0009
:100AA00030917B003901B4E08B2EB2E09B2E3430C4
:100AB00010F08A949A94383010F08A949A9476942C
:100AC00067948A94E1F726193709992021F0169541
:100AD00007959A94E1F7200F311F20937A00309305
:100AE0007B0028F43FEF30937A0030937B00323064
:100AF00008F4706871FF02C0B3E00DC0B091C4008B
:100B000000917100023838F0B395003A08F0B395BF
:100B1000B63008F0B5E09B2EB4E08B2E10917B0030
:100B200000917A0024E0169507952A95E1F70819B7
:100B3000120928F0B02FB250B12FB20910F402E020
:100B400010E0980126C020917A0030917B00390195
:100B5000769467946694669466942619320906958D
:100B60000695200F321D20937A0030937B0032309F
:100B700008F07F7704E036952795369527952695DA
:100B80002695201B10F0223008F422E08901909075
:100B9000C40060FDFECFE0908B00F0908C0061609F
:100BA000B9B7B061B9BF380177FD41C07694679499
:100BB00000938B0010938C00B92DB330E1F0B0FDA1
:100BC00004C0060D171D930106C0000F111F02502F
:100BD000120922E030E0B92DB33068F020938D0087
:100BE00030938E00009387001093880060928900F4
:100BF00070928A003AC000938D0010938E0020936B
:100C00008700309388006092890070928A0071FF9B
:100C10000DC0BFE0B0938D0020928E00B09389008C
:100C200020928A00B0938B0020928C001EC06694A4
:100C300000938B00B92DB33091F0B0FD03C0060DC9
:100C4000262D03C0000F025022E0B92DB33038F03A
:100C500020938D00009387006092890006C0009366
:100C60008D00209387006092890000917C0002FD36
:100C70000350013029F495FD0AC0B6E0B7B909C0A8
:100C8000023019F4B7E0B7B904C095FDF6CFB0E073
:100C9000B7B90091A200000F10F4BBE60B27009338
:100CA000A20060FDFECFB2E0B0936E006160B9B704
:100CB000B061B9BFB72FB670D1F020917A003091F2
:100CC0007B00369527953695279571FF02C0B0E4D5
:100CD0003B0FF8940CB51DB5020F131F1BBD0ABDC9
:100CE0006160B0E1B8BFB9B7B061B9BF7894089599
:100CF000606120927D0020E067FD20E206C0606117
:100D000020927D0020E267FD20E001E011E077FD08
:100D100011C0B72FB67009F06F7E14E100917B000F
:100D2000069509F403950F3008F00FE071FF02C03B
:100D300004E114E160FD0FC0B0917D00BB2359F0C8
:100D400071FF06C0B0916E00BA95B0936E0011F4B9
:100D5000706247C0ABDFB0B7B77FB0BFB8B1B0B754
:100D6000B860B0BFB0917D00B395B0937D00B8B1CD
:100D700077FD06C0B1E071FDB3E0BA95F1F7B8B107
:100D8000B072B21709F022C071FF05C003950117B8
:100D900008F00A95CFCF64FD05C00395011708F050
:100DA000B4CFC8CF6F7EF8943CB56DB470907A0024
:100DB00080907B00370D681C6BBC3ABD6160B0E170
:100DC000B8BFB9B7B061B9BF78949FCFB0916D008B
:100DD000B13008F49ACF64FD98CF0A9509F0AACFF4
:100DE0007F7D20918D0030918E00F894B0E1B8BFE6
:100DF0000CB51DB5020F131F1BBD0ABDE090870087
:100E0000F09088006160B9B7B061B9BF7894B72F2E
:100E1000B67039F0B0916D0072FFB395B0936D006C
:100E200009C075FF07C067FD05C064FD03C0BF9121
:100E3000BF91EAC4089500E063FF03C064FF01C0EE
:100E400001E0F89410917100B7E01B9F212D102D47
:100E50007894200F26951795269517952695179522
:100E600010937100183718F4B8E7B093710000912F
:100E70007100B09172000B1720F060629598AC98E9
:100E8000C09860FDFECFE0908900F0908A0061601C
:100E9000B9B7B061B9BF0895B2E095FD0AC0F89442
:100EA000B0937C00AD9A949862FF01C0C09A789488
:100EB000F4C0F894B0937C00AD9AAB9862FF01C087
:100EC000959A7894EAC0B3E082FF24C095FD11C0E2
:100ED00002E0F894B0937C00E0E8F0E00093B10009
:100EE000C098AB9A62FF02C0AC9A01C0AD987894EA
:100EF000D4C002E0F894B0937C00E0E8F0E0009306
:100F0000B1009598949A62FF02C0AC9A01C0AD9866
:100F10007894C3C095FD0BC0F894B0937C00EAE6CA
:100F2000F0E0C09862FF01C0AC9A7894B6C0F89423
:100F3000B0937C00EAE6F0E0959862FF01C0AC9ABD
:100F40007894ABC0B4E095FD0AC0F894B0937C00EF
:100F5000949AAB9862FF01C0AC9A78949EC0F894C2
:100F6000B0937C00AB9A949862FF01C0AC9A7894DD
:100F700094C0B5E082FF24C095FD11C001E0F89453
:100F8000B0937C00E6E7F0E00093B100AC98AD9A36
:100F900062FF02C0959A01C0949878947EC004E0E4
:100FA000F894B0937C00EAE8F0E00093B100AC98CC
:100FB000AD9A62FF02C0C09A01C0AB9878946DC030
:100FC00095FD0BC0F894B0937C00E4E6F0E0AC989B
:100FD00062FF01C0959A789460C0F894B0937C0049
:100FE000E0E7F0E0AC9862FF01C0C09A789455C089
:100FF000B6E095FD0AC0F894B0937C00AB9AAD982A
:1010000062FF01C0959A789448C0F894B0937C0030
:10101000949AAD9862FF01C0C09A78943EC0B1E046
:1010200082FF24C095FD11C004E0F894B0937C00C9
:10103000EAE8F0E00093B1009598949A62FF02C04C
:10104000C09A01C0AB98789428C001E0F894B0939E
:101050007C00E6E7F0E00093B100C098AB9A62FF35
:1010600002C0959A01C09498789417C095FD0BC062
:10107000F894B0937C00E0E7F0E0959862FF01C03F
:10108000C09A78940AC0F894B0937C00E4E6F0E04B
:10109000C09862FF01C0959A78946F7D089523E609
:1010A00030E0F9012092B1009598AC98C098949ADC
:1010B000AD9AAB9A6B7F0895A2EBB0E00FEF0D9362
:1010C0000D930D930D9303E00D9304E00D930AE04F
:1010D0000D9303E00D9301E00D9301E00D93AEEB52
:1010E000B0E001E00D930FEF0D930D930D930D9371
:1010F0000D9303E00D930FEF0D930FEF0D930D93F1
:1011000005E20D9300ED0D930AEF0D930AEF0D9399
:1011100004E00D930FEF0D9301E00D9300E00D93AC
:101120000AE70D930FEF0D9300E00D9301E00D938F
:1011300000E00D9303E00D9300E00D9308952091DE
:10114000B9008B7F233009F48460B091BA00B330CA
:1011500019F09F7DB1FD90629F7BB091BB00B1FD06
:101160009064223011F0886001C0877F08950A954D
:10117000E00FF21DB4910895ECE1F0E00091B200AF
:10118000F6DFB093D700ECE1F0E00091B300EFDFC1
:10119000B093D800EAE2F0E00091B800E8DFB09345
:1011A000D9000091B800023008F402E00093730007
:1011B000B091CE000FEFB23009F400EAB33009F479
:1011C00002E800937200E8E3F0E00091D500CFDF81
:1011D000B093A000089508952091C8003091C900EF
:1011E000B091BA00B33009F43E5097FF02C020E03E
:1011F0003FEFB32FB21B6B2EB25810F4B2E86B2E38
:1012000000E00395609EB12DBD57D8F30093AC006C
:1012100008959068E1DF0CDA20E030E0B0E16B2E59
:1012200003DAB09196002B0F321D6A94C9F7B4E02F
:1012300036952795BA95E1F7822E9F77CDDF0895F1
:10124000F894E3E0F0E0B9E0B7BFB491B078C1F34F
:10125000F894A895B1B5B861B1BDB0E0B1BDB4E046
:10126000BEBFBFE5BDBF1BDFB0E0B8BBB1E1B7BBE0
:10127000B8E2B5BBB8E3B4BBB0E1B2BBB0E3B1BB5D
:101280002224A0E0B0E02D92AA31E9F7A0E6B0E078
:101290000FEF2D920A95E9F7B1E0B093A2000CDFB1
:1012A000EBD2B6B1B460B6B90091CA000093AD00FC
:1012B000B1E0B0936A00F894BFD9C9D9B9D9CAD9F5
:1012C000B7D9CBD9B5D95FD3B7D9B6D9B3D9F894F3
:1012D0000AEF1AEFA0B396FDA095A2FF1FC01A95C2
:1012E000C9F70A95B1F7E0E0FCE1B591B43E39F4F5
:1012F000B591B03E21F4B591BF3F09F40CC0E0E0D8
:10130000F395F395B591B83F49F4B591B43931F4FB
:10131000B591BA3A19F4EE27F695099410DF2CDF4F
:101320005ADF5ADF0091CA000093AD00B8DEB2E088
:10133000B3BFB2E0BEBDB2E0B5BDB1E5B8BFB9BFA5
:10134000B0B7B77FB0BFB8B1B0B7B860B0BF6AD9F7
:101350007894FEDA20927000B3E096FDB2E0B5BF5B
:10136000B0E4BBBFBB27B064BABF8D7F65D96260F4
:1013700033E02CE0B0919500BB2321F42CE03A95AA
:1013800009F4A5CF55D980FFA2CF8E7FB0919600EA
:10139000B23078F3B92FBF71009198000093970095
:1013A000B0939800B01729F72A9521F76D7FB3E025
:1013B00096FDB2E0B5BFBB27B064BABF8D7FB091D8
:1013C000D400BB2321F48062B92FB0709B2F8F7B98
:1013D000209267002FD985FF05C0B0916700BA3011
:1013E00008F0806421D902E085FF01C000E0B091DF
:1013F0009600B017B8F3F8942AD929D928D9789447
:101400001BD920928600B091BA00B33009F474C0A1
:101410000BD9B091BE00B13008F46EC0B0916A0033
:10142000B13008F469C085FD18C0B0919600BF3F87
:1014300008F462C0F89414D97894FCD8B09196005E
:10144000B130C0F7F89403D9F1D801D97894F2D823
:10145000B0919600BF3FB0F3C8C2B8E09B2E906831
:10146000F894BADE7894E6D8F8949F77B5DE809049
:101470009600B0919600BF37789408F445C0D2D852
:10148000F894EED878949A9451F7C3DEB82DB550FD
:10149000B093C900D1D8F8941CD27AD27894BAE02B
:1014A0009B2E9068F89498DE7894C4D8F8949F772F
:1014B00093DE80909600B0919600BF37789478F7CD
:1014C000B1D8F894C4D8B2D8C2D878949A9449F7CD
:1014D000A0DEB82DBB5FB093C800AED8F894F9D1A8
:1014E00066D27894A7D8F89477DE7894B091960075
:1014F000BF3F08F498CF79C200919600B091860062
:101500000B1710F00093860095D801E0B091BA0057
:10151000B35009F405E0B0919600B01708F073CF0E
:10152000F8949ED89DD89CD8789486D820926A004A
:1015300020926B0020926C00B0916B00B395B09339
:101540006B00BF3F71F5B0916C00B395B0936C0028
:10155000B091CC0009E1BA9559F002E3BA9541F097
:101560000DE7BA9529F00AEFBA9511F020926C00B8
:10157000B0916C00B017A8F092DD54D8B0916C0017
:10158000BA95B0936C0020926B00B091CB00B093F1
:10159000AD00F89465D87894B091CA00B093AD00CE
:1015A00049D844D8B0916800BB2319F485FF01C025
:1015B0008ECE01E085FD01C006E0B0919600B01727
:1015C00008F4BACFB091BA00B35009F033D8B09153
:1015D0006800BB2309F47BCEF89461DD20926100A2
:1015E0002092620020926300522C2092640020928C
:1015F000A1007894B091B700BB0FB0939F002092E8
:101600007E0020927F002092800020928100209214
:1016100082002092AA0060E070E020927100B8E0A1
:10162000B093AA007061FED7B2E074FDB1E0B7B923
:10163000B6B1B068B064B6B9B6B1B6FDFDCF04B10D
:1016400015B1B6B1BF77B6B9112309F00FEF00930A
:10165000AB0080D9B8E0B093AA00706170DDF89457
:10166000BFEFB0939B00BFD9B0916100B0939B00D6
:10167000B0939C00B0939D007894B1E0B09361006A
:10168000B09363005B2EB0936400B093A400B0915C
:101690009A00B093A300B091BA00B33019F49F7DC3
:1016A00087FD90627160726020926D00A1DCB7DCF2
:1016B000B3D9B8D9B1D9B6D9AFD921DB4ED8BBDBB4
:1016C000EBDBB0D915DB66FD49D877FF01D977FD93
:1016D0002FD9B1DBF8DBA6D912DB66FD61D8ABDB15
:1016E00031DCA0D905DB66FD95D8A5DB42DC9AD9B3
:1016F00006DB66FDBFD89FDB7BDC94D9F9DAB2E06C
:1017000074FDB1E0B7B9B6B1B068B064B6B993DBF7
:1017100086DC88D91FD971FF21C0B0919E00B0939B
:101720009B00B0939C00B0919A00B093A300B1E0ED
:10173000B093A40018E12CE0B0916D00B11740F017
:101740007D7F746020936F00BFEFB0939B0006C055
:10175000B0919600B13008F0B0CF60C072FF11C0F8
:1017600067FD0FC0B0916F00BA9519F47B7F786068
:10177000A4CFB0936F00B0919600B13008F09DCF28
:101780004DC020927000B091990002E81091D600EF
:10179000112309F003E0B01708F040C085FF04C032
:1017A000B0916800BB23D1F1B091BA00B33081F49D
:1017B00095FD03C087FD04C00BC087FF01C008C0B2
:1017C00067FD06C06068B0919E00B0939B008ACF11
:1017D00000EF67FF05C0B0919E00B0939B0000E250
:1017E000B0917B00B01708F468CF67FF17C06F7720
:1017F0009F7D87FD90627460B2E1B0936F00B091FD
:101800009E00B0939B0059CFB0917000B395B093F8
:101810007000B0919600BB2309F002C020927000C6
:10182000F8943DDC8090B900B2E0B093B90087DC59
:101830008092B900209261002092620020926300A1
:10184000522C2092640020929F0060E070E0789417
:10185000F1D625DC0091D600002319F0959AAC9AB8
:10186000C09AB6B1B460B6B985FF05C0B09170003A
:10187000B43008F02CCD5CCEEDE0F0E023D00A359A
:1018800009F01BC0EEE0F0E01DD0053A09F015C0EC
:101890003AE0A2EBB0E0E3E0F0E014D00D93319633
:1018A0003A95D9F739E1AEEBB0E0EFE0F0E00AD0DD
:1018B0000D9331963A95D9F702C0FEDB0AD0E8E2E3
:1018C000F0E00895E199FECFEEBBFFBBE09A0DB3C7
:1018D00008951ED03AE0A2EBB0E0E3E0F0E00D9115
:1018E0000FD031963A95D9F739E1AEEBB0E0EFE0A1
:1018F000F0E00D9105D031963A95D9F712D00895C0
:10190000E199FECF0DBBEEBBFFBBE29AE19A0895D1
:10191000EDE0F0E00FEFF4DFEEE0F0E00FEFF0DFEE
:101920000895EDE0F0E00AE5EBDFEEE0F0E005EA37
:10193000E7DF08953091AE000091AF00313011F42F
:101940000093B600323011F40093B700333011F435
:101950000093B800343011F40093C400353011F412
:101960000093B900363011F40093D500373011F4EC
:101970000093CE00383011F40093BA00393011F4DE
:101980000093BB00089525E057D62A95E9F70895FE
:101990005ED660D662D664D649D659D65BD65DD6B9
:1019A0005FD644D654D656D658D65AD6089558D669
:1019B00054D650D64CD63AD653D64FD64BD647D619
:1019C00035D64ED64AD646D642D608958090AE0039
:1019D0009090AF003CD63BD63AD628D68A94D1F721
:1019E0003FD624D69A94E1F70895F894D1DF7894FD
:1019F000CADFC9DFB1E0B093AE00B1E0B093AF0091
:101A00002092B000F894E2DF7894B5E06B2E7090ED
:101A1000960012D6B09196007B16C9F7B13018F037
:101A2000BF3F40F107C086DFF89453DFB1DFB8E075
:101A3000B1BDA9DF6A9459F7B091B000B395B093E6
:101A4000B000B33008F4DECF9EDFB091AF00B395A5
:101A5000B093AF00F894B091AE00BA95EEE3F0E029
:101A6000EB0FF21D049178940395B091AF00B0177D
:101A700008F4C6CF88DF87DFB091AE00B395B0938E
:101A8000AE00B091AE00BA3008F4B7CF15DBF894D1
:0A1A900020DFB8E0B1BD77DFD3CB53
:00000001FF
